:0A234E000001020203030404050568
:100FB800E4F565F564F563F562C209C206C208C2C4
:100FC8000712221F120A337E1A7F008E0A8F0B75B2
:100FD800121A75131275081A75091C75101A7511ED
:100FE8005175161A75177FEE54E070030210FF75DD
:100FF80066007567808E688F69C374A99FFF741A2D
:101008009ECF2402CF3400FEE48F618E60F55FF539
:101018005EF55DF55CF55BF55AAF61AE60AD5FAC52
:101028005EAB5DAA5CA95BA85AC31206B75026E559
:1010380067255DF582E566355CF58374CDF0E55D81
:101048002401F55DE4355CF55CE4355BF55BE4357E
:101058005AF55A80C4E4F55DF55CF55BF55AAF6165
:10106800AE60AD5FAC5EAB5DAA5CA95BA85AC3126B
:1010780006B75031AE5CAF5DE5692FF582E5683E95
:10108800F583E0FDE5672FF582E5663EF583EDF033
:10109800EF2401F55DE43EF55CE4355BF55BE43592
:1010A8005AF55A80B985660A85670B74002480FF53
:1010B800741A34FFFEC3E5139FF513E5129EF5126B
:1010C800C3E50D9FF50DE50C9EF50CC3E50F9FF5E7
:1010D8000FE50E9EF50EC3E5099FF509E5089EF597
:1010E80008C3E5119FF511E5109EF510C3E5179F9C
:1010F800F517E5169EF516D2E843D82090E668E085
:101108004409F090E65CE0443DF0D2AF90E680E020
:1011180020E105D20A121F6F90E680E054F7F053E1
:101128008EF8C20930070512080FC20730092912C4
:1011380023CA5024C20912213E20061690E682E0F6
:1011480030E704E020E1EF90E682E030E604E020BA
:0D115800E0E4121F9E1223CC1215DE80C7AA
:10080F0090E6B9E070030208C014700302093D249A
:10081F00FE70030209C024FB70030208BA147003B0
:10082F000208B414607314607624056003020A1F73
:10083F001223CE4003020A2B90E6BBE024FE602277
:10084F0014603324FD601114602224067048E50AF9
:10085F0090E6B3F0E50B8037E51290E6B3F0E513C1
:10086F00802DE50C90E6B3F0E50D8023E50E90E6C4
:10087F00B3F0E50F801990E6BAE0FF121FCAAA067F
:10088F00A9077B01EA494B600DEE90E6B3F0EF90BC
:10089F00E6B4F0020A2B020A241222CC020A2B120F
:1008AF0023AA020A2B121BBC020A2B1222BA020A1B
:1008BF002B1223D04003020A2B90E6B8E0247F606E
:1008CF001514601924027063A206E43325E0FFA219
:1008DF0008E4334F8041E490E740F0803F90E6BC5E
:1008EF00E0547EFF7E00E0D394807C0040047D01C5
:1008FF0080027D00EC4EFEED4F244EF58274233EB8
:10090F00F583E493FF3395E0FEEF24A1FFEE34E689
:10091F008F82F583E0540190E740F0E4A3F090E676
:10092F008AF090E68B7402F0020A2B020A2412233B
:10093F00D24003020A2B90E6B8E024FE6016240290
:10094F006003020A2B90E6BAE0B40105C206020A60
:10095F002B020A2490E6BAE0705590E6BCE0547E74
:10096F00FF7E00E0D394807C0040047D0180027DF7
:10097F0000EC4EFEED4F244EF58274233EF583E4DA
:10098F0093FF3395E0FEEF24A1FFEE34E68F82F55F
:10099F0083E054FEF090E6BCE05480131313541F11
:1009AF00FFE0540F2F90E683F0E04420F0806D803D
:1009BF00641223D4506690E6B8E024FE6019240236
:1009CF00705A90E6BAE0B40104D206804F90E6BAAE
:1009DF00E064026047803E90E6BCE0547EFF7E00FC
:1009EF00E0D394807C0040047D0180027D00EC4EBA
:1009FF00FEED4F244EF58274233EF583E493FF33CF
:100A0F0095E0FEEF24A1FFEE34E68F82F583800898
:100A1F00120080500790E6A0E04401F090E6A0E0BD
:030A2F004480F010
:010A320022A1
:030033000219FCB3
:0419FC0053D8EF329B
:10221F00758CE0758AC0E58954F04401F589758E97
:08222F0003D28CD2A9D2AF2228
:03000B00021AAB2B
:101AAB00C0E0C0F0C083C082C0D075D000C000C001
:101ABB0001C002C003C004C005C006C007758CE09E
:101ACB00758AC0D28CE47F607EEAFDFCAB55AA54CC
:101ADB00A953A852C31206B75019AF55AE54AD5304
:101AEB00AC52EF2401F555E43EF554E43DF553E4D7
:101AFB003CF552E47F01FEFDFCAB55AA54A953A85B
:101B0B0052C31206B77008E5A054F02534F5A0E5D2
:101B1B002A2401FFE43529FEE4FCFDAB55AA54A9A8
:101B2B0053A852C31206B7700553A0F0C28CD0074E
:101B3B00D006D005D004D003D002D001D000D0D035
:091B4B00D082D083D0F0D0E0324A
:03003B00021B5451
:101B5400C0E0C083C082C0D075D000C006C00730CA
:101B6400C041C2C085C114052EE52E7002052DD3D7
:101B7400E52E94F4E52D648094814006752D00755E
:101B84002E00AE2DAF2EEE90F800F0AE2DAF2EEF5E
:101B9400A3F0AE2DAF2E74012FF58274F83EF583B9
:101BA400E514F030C105C2C185C114D007D006D0F8
:081BB400D0D082D083D0E032D2
:03002300021C1BA1
:101C1B00C0E0C083C082C0D075D000C007309836FA
:101C2B00C298859915052CE52C7002052BD3E52C54
:101C3B00940EE52B648094804006752B00752C0068
:101C4B00AF2C90E7F0EFF0AF2C74F02FF582E4346B
:101C5B00E7F583E515F0D007D0D0D082D083D0E064
:011C6B003246
:101A000012010002000000401816511600000102E9
:101A100000010A0600020000004001000902350032
:101A200001010080FA0904000005FF00000007051D
:101A30000102400000070582020002000705810242
:101A400040000007058602000200070508020002A8
:101A50000009022E0001010080FA0904000004FFC1
:101A60000000000705010240000007058202400057
:101A70000007050202000200070581024000000481
:101A800003090410035100480059002D004300438E
:101A9000004400160351004800590032003700206E
:0B1AA0000020002000200020000000BB
:10136A0060802800030A0303020203070000000248
:10137A00000002000B2A0A121014101000000000CC
:10138A000000003F020A03030303030700000002F0
:10139A00000002000B2A120A1014101000000000AC
:1013AA000000003F032D03030303030700000002AC
:1013BA00000002000B2A0A1210141010000000008C
:1013CA000000003F030A0A0A0A0A0A07000000028C
:1013DA00000002000B2A120A10141010000000006C
:1013EA000000003F60242887000000000000000081
:1013FA0000000000000000000000000000000000E3
:10140A000000000000000000000000004728808063
:06141A00000010CA4E00A4
:1016A10090E60174CAF090E6F574FFF0902880E0AE
:1016B10090E6F3F0902881E090E6C3F0902882E074
:1016C10090E6C1F0902883E090E6C2F0902885E092
:1016D10090E6C0F0902886E090E6F4F075AF0774CC
:1016E10028F59A7400F59B759DE4E4F59EFF90E65C
:1016F1007BE090E67CF00FBF80F490E67174FFF020
:10170100F5B490E672E04480F043B680000000E456
:1017110090E6C4F000000090E6C5F0902887E090C4
:10172100E6C6F0902888E090E6C7F0902889E0901E
:10173100E6C8F090288AE090E6C9F090288BE09006
:10174100E6CAF090288CE090E6CBF090288DE090EE
:0B175100E6CCF090288EE090E6CDF092
:01175C00226A
:03004300021800A0
:0300530002180090
:101800000222370002227D000222670002224F00DE
:10181000021E6B00021D7F000223D6000223D700A8
:101820000223D8000223D900021DBC00020DFC00D7
:101830000223DA000223DB00021D3C0002126D00CD
:101840000223DC000223D7000223DD000223DE0096
:101850000223DF000223E0000223E1000223E20072
:101860000223E3000223D7000223D7000223D7007C
:101870000223E4000223E5000223E6000223E7003E
:101880000223E8000223E9000223EA000223EB001E
:101890000223EC000223ED000223EE000223EF00FE
:1018A0000223F0000223F1000223F2000223F300DE
:0818B0000223F4000223F500FD
:101F9E0090E682E030E004E020E60B90E682E0304E
:101FAE00E119E030E71590E680E04401F07F147E01
:0C1FBE0000121C6C90E680E054FEF02243
:10213E0090E682E044C0F090E681F0438701000013
:04214E00000000226B
:101F6F00300A0990E680E0440AF0800790E680E0AE
:101F7F004408F07FDC7E05121C6C90E65D74FFF068
:0F1F8F0090E65FF05391EF90E680E054F7F02278
:021FCA00A90765
:101FCC00AE16AF178F828E83A3E064037017AD013A
:101FDC0019ED7001228F828E83E07C002FFDEC3E88
:091FEC00FEAF0580DF7E007F00DE
:011FF50022C9
:101C6C008E6E8F6F90E600E054187012E56F2401B1
:101C7C00FFE4356EC313F56EEF13F56F801590E628
:101C8C0000E05418FFBF100BE56F25E0F56FE56E13
:101C9C0033F56EE56F156FAE6E7002156E4E600506
:061CAC0012215280EE221D
:102152007400F58690FDA57C05A3E582458370F9A0
:01216200225A
:10142000C18202311040C100014800C105C104045D
:101430004E00000000014500012500043F000000AF
:0A1440000004370000000001350031
:100A330090E600E054E74410F0000000000000904E
:100A4300E61074A0F000000090E60B7401F090E64D
:100A53001274E0F0000000E490E613F00000009050
:100A6300E61474E2F000000090E61574A0F00000B4
:100A73000090E6D27402F090E6047480F000000067
:100A83007402F00000007406F00000007408F00027
:100A93000000E4F00000001216A190E6187408F0BC
:100AA30000000090E619F000000090E61AF0000044
:100AB3000090E61BF0000000E490E670F075B2FFD2
:100AC3007580FF90E671F075B47F75A0FF90E672B4
:100AD300F075B6BF75B13FC28CD28753A0FD122308
:100AE300BA90E61074A0F000000090E611F0000048
:100AF3000090E65EE04408F0000000E490E68DF02C
:100B030000000090E65EE04404F0000000E490E79B
:100B1300C0F090E7C4F0A3F0A3F0A3F090E7F0F0E7
:100B230090E68F7440F000000090E65EE04440F0F1
:100B33000000007E027F0090F800E4F0A3DFFCDEFB
:100B4300FA90E6987402F0000000E490E699F00051
:100B530000007E027F0090F800E4F0A3DFFCDEFAE1
:100B630090E65EE04480F0000000E490E69CF00034
:100B7300000090E69DF00000007F9AFE122362754C
:100B830027007528B4754901754A9075311075327F
:100B9300B8754C06754D2C1223B290E67AE054FEDC
:100BA300F0E4FD7F901222DE7F647E00121C6C7DD8
:100BB300FF7F421222DE7F647E00121C6C7D827FE7
:100BC3004E1222DE7536FF43B108E4F53D90E7820D
:100BD300E536F090E781E53DF01217E9E4F52BF5F2
:100BE3002C1220A1E4F52DF52E1223BA1221A97F90
:100BF300887E131221711221A97F887E131221711D
:100C03001221A97F887E1312217112232A12175DE4
:100C13007F55121DF87F887E13122171D2F9C2F815
:0C0C2300E4F54590E7C0E545F053A0F76C
:010C2F0022A2
:0E230200EF2401FBE43EFA7D047F480221E750
:100C3000E53DC313FFC374809FF572E53DD3940077
:100C400040067536FF43B108E53D700353B1F77EAA
:100C5000297F0B12230290290CE090E7C1F0902924
:100C60000DE090E7C2F09028EB74E5F07A287BEB7A
:100C70007D017F411222037E007F0A7D007B017A85
:100C8000E779401207157A297B0B7D027F411221FB
:100C9000E790290BE0FEA3E07C002400FFEC3EFE81
:100CA000E48F718E70F56FF56E7F097E3DFDAB713F
:100CB000AA70A96FA86E120652780D1206DBEF24F7
:100CC00090F571EE34E8F570ED34FFF56FEC34FF1C
:100CD000F56EE4FB7A01F9F8AF71AE70AD6FAC6EF2
:100CE000121CF890E7CCEFF0E4FB7A01F9F8AF7151
:100CF000AE70AD6FAC6E121CF890E7CDEBF09028A3
:100D0000EB7450F0A3742EF07A287BEB7D027F41C8
:100D10001222039028EB74EEF07A287BEB7D017FA2
:100D2000411222037E007F0A7D007B017A29790B24
:100D30001207157A297B0B7D027F411221E790294A
:100D40000BE0FEA3E07C002400FFEC3EFEE48F718C
:100D50008E70F56FF56E9028EB7450F0A3740FF061
:100D60007A287BEB7D027F41122203E47FCD7E5502
:100D7000FDFCAB71AA70A96FA86E120652780D1215
:100D800006DBEF24FEF571EE3448F570ED34FFF527
:100D90006FEC34FFF56EE4FB7A01F9F8AF71AE70D9
:100DA000AD6FAC6E121CF890E7CEEFF0E4FB7A0169
:100DB000F9F8AF71AE70AD6FAC6E121CF890E7CF62
:100DC000EBF09028EBE536F07A287BEB7D017F2174
:100DD0001222039028EB7402F0A37480F07A287B2F
:100DE000EB7D027F28122203E49028EBF0A3E5724A
:0C0DF000F07A287BEB7D027F28022203B2
:1015DE00E5512401F551E43550F550E4354FF54F02
:1015EE00E4354EF54EE47FE87E03FDFCAB51AA5088
:1015FE00A94FA84EC31206B7700F9028EBF07A28A9
:10160E007BEB7D017F481222037FA07E867D017CCD
:10161E0000AB51AA50A94FA84EC31206B7700E12B6
:10162E000C3090E6907402F0E490E691F07F407EEC
:10163E000D7D037C00AB51AA50A94FA84ED31206C4
:10164E00B7400CE4F551F550F54FF54E121F0B3027
:10165E00014075450190E7C0E545F0E5B130E7037F
:10166E002005F8121515C201E4F54590E7C0E545D1
:10167E00F01221A97F887E131221711221A97F8871
:10168E007E131221711221A97F887E1312217112ED
:03169E00232A22DA
:0223CA00D3221C
:0223CC00D3221A
:0223CE00D32218
:101BBC0090E680E030E73A00000090E6207402F0F6
:101BCC00000000E490E621F000000090E62474028E
:101BDC00F0000000E490E625F000000090E626748A
:101BEC0002F0000000E490E627F0000000D2028032
:101BFC0016000000E490E620F000000090E621744E
:0F1C0C0040F0000000C20290E6BAE0F546D32295
:1022BA0090E740E546F0E490E68AF090E68B04F079
:0222CA00D3221D
:0823AA0090E6BAE0F526D3220B
:1022CC0090E740E526F0E490E68AF090E68B04F087
:0222DC00D3220B
:0223D000D32216
:0223D200D32214
:0223D400D32212
:10008000E4F56AF56B90E6B9E01206EF00B1B30053
:10009000E9B50266B6029EBB02E5BC038EC103460B
:1000A000C2040CC5042BC60460CA04A1CB00000521
:1000B00009E490E68AF090E68BF090E6A0E020E17B
:1000C000F990E68BE0F56AE4F5B390E60174CAF0C6
:1000D000D20100000090E6047480F0000000740279
:1000E000F0000000E4F002050BE490E68AF090E6F0
:1000F0008BF090E6A0E020E1F990E68BE0F56AD382
:10010000943F4024E4F56B7440256BF582E434E7BA
:10011000F583E0FF74AB256BF582E43428F583EFBB
:10012000F0056BE56BB440DF7F8A7E00122362909E
:1001300028ABE0FF7E0012236B9028ABE0FF7E002F
:100140001223749028ABE0FF7E0012237D9028AC30
:10015000E075F004A4FFAEF01223869028ACE075A1
:10016000F004A4FFAEF012238F9028ACE075F004E9
:10017000A4FFAEF01223989028B0E0C3940250136D
:100180009028CCE090E6C07005744EF08016749C08
:10019000F080119028CCE090E6C07005749FF0804C
:1001A00003749DF09028CEE0F53E9028CBE0F53C1E
:1001B0009028CFE0F5479028D9E0F53BA3E0FEA3D7
:1001C000E07C002400F524EC3EF5239028B1E0F516
:1001D00033E53370037533019028B6E0FEA3E07C6D
:1001E000002400F528EC3EF527A3E0FEA3E0240060
:1001F000F54AEC3EF5499028B2E0FEA3E02400F574
:1002000032EC3EF531A3E0FEA3E02400F54DEC3ED8
:10021000F54C9028BCE0FEA3E02400F544EC3EF54C
:10022000439028BAE0FEA3E02400F530EC3EF52F21
:100230009028E0E0540FF535E4FD7F901222DE9027
:1002400028ACE0FCA3E0FDA3E0FEA3E0F5428E4174
:100250008D408C3FE542F542E541F541E540F540F2
:10026000E4F53F02050BE4F56B74AB256BF582E416
:100270003428F583E0FF7440256BF582E434E7F51C
:1002800083EFF0056BE56BB440DF000000E490E61F
:100290008AF000000090E68B7440F002050BE490B9
:1002A000E68AF090E68BF090E6A0E020E1F978EBAA
:1002B0007C287D017B017AE679BC7E007F011205F6
:1002C000DD90E6BEE0FF7E0078EC7C287D017B01BE
:1002D0007AE779401205DD90E6BAE0C313FF90E6B5
:1002E000BEE0048059E490E68AF090E68BF090E658
:1002F000A0E020E1F978EB7C287D017B017AE679AA
:10030000BD7E007F011205DD78EC7C287D017B013C
:100310007AE679BC7E007F011205DD90E6BEE0FF43
:100320007E0078ED7C287D017B017AE7794012051B
:10033000DD90E6BAE0C313FF90E6BEE02402FD7A4A
:10034000287BEB02050490E74074F4F0A37417F0E7
:10035000A3740CF0A37426F0A37407F0A374EEF05A
:10036000A37401F0A37403F0A37453F0300205E406
:10037000A3F0800690E74974FFF0000000E490E6E7
:100380008AF000000090E68B740AF002050BE490FE
:10039000E68AF090E68BF090E6A0E020E1F990E6A6
:1003A0008BE0F56AC298D39400500302050B90E7E6
:1003B00040E0940A5007E02430FF12231090E740F9
:1003C000E0B40A057F6112231090E740E0B40B050A
:1003D0007F6212231090E740E0B40C057F63122384
:1003E0001090E740E0B40D057F6412231090E740C1
:1003F000E0B40E057F6512231090E740E0640F60C3
:100400000302050B7F6612231002050B7AE77B407F
:100410007D047F481221E7000000E490E68AF000A6
:10042000000090E68B7404F002050BE490E68AF07D
:1004300090E68BF090E6A0E020E1F990E68BE0F505
:100440006AD39401500302050B90E741E0FD7F421F
:100450001222DE90E740E0FD7F4E1222DE02050B05
:1004600090E6BCE090290BF07A297B0B7D017F5050
:100470001222037A297B0B7D017F5012220390E622
:10048000BEE0FD7AE77B407F501221E7E490E68AE8
:10049000F000000090E6BEE090E68BF000000080E7
:1004A0006AE490E68AF000000090E68BF00000001D
:1004B00090E6A0E020E1F990E6BCE0D39407404B41
:1004C00078EB7C287D017B017AE679BC7E007F0198
:1004D0001205DD90E6BEE0FF7E0078EC7C287D0111
:1004E0007B017AE779401205DD90E6BEE004FD7AF3
:1004F000287BEB7F5012220390E6BEE004FD7A28B1
:0C0500007BEB7F501222038002D322C349
:01050C0022CC
:10223700C0E0C083C082D2075391EF90E65D74017E
:08224700F0D082D083D0E03218
:10226700C0E0C083C0825391EF90E65D7404F0D064
:0622770082D083D0E032AA
:10227D00C0E0C083C0825391EF90E65D7402F0D050
:06228D0082D083D0E03294
:101E6B00C0E0C083C08285100C85110D850D828565
:101E7B000C83A37402F085080E85090F850F8285EC
:101E8B000E83A37407F05391EF90E65D7410F0D0BE
:061E9B0082D083D0E0328A
:10224F00C0E0C083C082D2095391EF90E65D74085D
:08225F00F0D082D083D0E03200
:101D7F00C0E0C083C08290E680E030E72085080C89
:101D8F0085090D850D82850C83A37402F085100ED5
:101D9F0085110F850F82850E83A37407F05391EF82
:0D1DAF0090E65D7420F0D082D083D0E03249
:0123D60032D4
:0123D70032D3
:0123D80032D2
:0123D90032D1
:101DBC00C0E0C083C08290E65EE054FBF0000000FF
:101DCC0090E68F7440F0000000752B00752C00908D
:101DDC00E7F0E4F05391EF90E65FE04404F090E616
:0C1DEC005EE04404F0D082D083D0E032EE
:100DFC00C0E0C0F0C083C082C0D075D000C000C0BD
:0D0E0C0001C002C003C004C005C006C0073D
:100E190090E65EE054F7F090E6A1E020E1F990E772
:100E290080E0FF1206EF0E4E000E54010E63300EE5
:100E390097310EDB320F19330F4A340F75FE0F7FCE
:100E4900FF00000F84752200020F8490E782E0F50D
:100E59003690E781E0F53D020F847556007557011C
:100E690090E68DE0FFC3E5579F7480F8655698407A
:100E790003020F8474802557F582E434E7F583E093
:100E8900FF12231D0557E55770D6055680D290E706
:100E990081E07006758DB2020F8490E781E0B4019C
:100EA90006758D64020F8490E781E0B40206758DA2
:100EB900D9020F8490E781E0B40306758DE6020F2D
:100EC9008490E781E064046003020F84758DF30266
:100ED9000F8490E781E070061221A9020F8490E740
:100EE90081E0B40106122188020F8490E781E0B401
:100EF900020612204D020F8490E781E0B403051227
:100F090021C8807790E781E0F4707012232A806B02
:100F190075560075570190E68DE0FFC3E5579F743C
:100F290080F8655698505474802557F582E434E763
:100F3900F583E0FF1223100557E55770D905568050
:100F4900D590E781E0F46011E024B0FF1222A7E414
:100F5900FF1222A77F101222A790E7817440F07A2E
:100F6900E77B817D217F3C122203800F90E781E09E
:100F790024FF92058005752200D20300000090E647
:100F89008DE4F05391EF90E65FE04408F090E65E5F
:040F9900E04408F038
:100F9D00D007D006D005D004D003D002D001D000A8
:0B0FAD00D0D0D082D083D0F0D0E03252
:0123DA0032D0
:0123DB0032CF
:101D3C00C0E0C083C08290E65EE054BFF0000000BB
:101D4C0090E6987402F000000090E699E4F0000030
:101D5C0000F52DF52E90F800F0A3F05391EF90E6DE
:101D6C005FE04440F090E65EE04440F0D082D083E7
:031D7C00D0E03282
:10126D00C0E0C0F0C083C082C0D075D000C000C047
:0D127D0001C002C003C004C005C006C007C8
:10128A0090E65EE0547FF090E6A6E020E1F990E671
:10129A009CE0FE90E69DE07C002400F557EC3EF5CC
:1012AA0056E55764054556704D90FC00E0B4EE14BF
:1012BA00A3E0B4440FA3E0B4880AA3E07006A3E055
:1012CA0064336064755800755900C3E5599557E54C
:1012DA00566480F8E558648098504D74002559F595
:1012EA008274FC3558F583E0FF12231D0559E55930
:1012FA0070D8055880D4755800755900C3E55995BA
:10130A0057E5566480F8E558648098501B740025A8
:10131A0059F58274FC3558F583E0FF12231D0559EF
:10132A00E55970D8055880D400000090E69CE4F096
:10133A0090E69DF05391EF90E65FE04480F090E6EE
:05134A005EE04480F0AC
:10134F00D007D006D005D004D003D002D001D000F2
:0B135F00D0D0D082D083D0F0D0E0329C
:0123DC0032CE
:0123DD0032CD
:0123DE0032CC
:0123DF0032CB
:0123E00032CA
:0123E10032C9
:0123E20032C8
:0123E30032C7
:0123E40032C6
:0123E50032C5
:0123E60032C4
:0123E70032C3
:0123E80032C2
:0123E90032C1
:0123EA0032C0
:0123EB0032BF
:0123EC0032BE
:0123ED0032BD
:0123EE0032BC
:0123EF0032BB
:0123F00032BA
:0123F10032B9
:0123F20032B8
:0123F30032B7
:0123F40032B6
:0123F50032B5
:06144B008F6C8C6D8D6EAC
:10145100536C0753A0BF7F0A7E00122171E4F56F20
:10146100F570C374029570FFE56CA807088002C38C
:1014710013D8FC30E00543A020800353A0DF7F0A8E
:101481007E0012217143A0107F0A7E001221715348
:10149100A0EF7F0A7E001221710570E570700205D0
:1014A1006FC39403E56F6480948040B6E4F56FF5F3
:1014B10070C374099570FFE56EAE6DA807088005CD
:1014C100CEC313CE13D8F930E00543A020800353D7
:1014D100A0DF7F0A7E0012217143A0107F0A7E00E7
:1014E10012217153A0EF7F0A7E001221710570E570
:1014F100707002056FC3940AE56F6480948040B1F7
:1015010043A0407F0A7E0012217153A0BF7F0A7E53
:041511000002217142
:09236200AD07AC06E4FF02144BC8
:09236B00AD07AC067F0402144B1F
:09237400AD07AC067F0502144B15
:09237D00AD07AC067F0602144B0B
:09238600AD07AC067F0102144B07
:09238F00AD07AC067F0202144BFD
:09239800AD07AC067F0302144BF3
:1022DE009028EBEDF0EFC313FF7A287BEB7D010224
:0222EE002203C9
:1020C9009028EB7402F0A37480F07A287BEB7D02F0
:1020D9007F28122203E49028EBF0A3F07A287BEB07
:0720E9007D027F28022203A3
:1022A700E49028EBF0A3EFF07A287BEB7D027F3CEC
:0322B700022203FD
:102293009028EB7440F0A3EFF07A287BEB7D027F6C
:0422A3003C022203D4
:10175D007FAE1222A77F041222A77F101222A77F2D
:10176D00401222A77FB01222A77F811222A77F806D
:10177D001222A77FA11222A77FA61222A77FA8124D
:10178D0022A77F3F1222A77FAD1222A77F8B1222A5
:10179D00A77F301222A77FC81222A77FD31222A7BC
:1017AD00E4FF1222A77FD51222A77F801222A77FE6
:1017BD00D91222A77F221222A77FDA1222A77F0237
:1017CD001222A77F8D1222A77F141222A77FDB1270
:0C17DD0022A77F401222A77FAF0222A7A4
:021DF8008F6AF0
:101DFA00E4FF1222A77F101222A7E4F56CE56C24F7
:101E0A00B6FF1222A7E4FF1222A77F101222A7E42C
:101E1A00F56BAF6A122293056BE56BC3946040F2CF
:091E2A00056CE56CC3940240D480
:011E3300228C
:0E2163007FFC7E0812217112234A7FFC7E0849
:10217100EF7803C333CE33CED8F9FFEF4E6007EFCC
:072181001F70F81E80F5221B
:0123F60022C4
:0123F70022C3
:0123F80022C2
:0123F90022C1
:0423BA007580E32225
:101CB2007580E37F027E001221717580EA7F027EC9
:101CC200001221717580CE7F0A7E0012217175800B
:101CD200EC7F027E001221717580CE7F0A7E001297
:101CE20021717580C77F027E001221717580E37FAA
:061CF200027E00022171D8
:101F0B007580E37F027E001221717580EA7F027E6D
:101F1B00001221717580CE7F027E001221717580B7
:101F2B00C77F027E001221717580E37F027E000263
:021F3B00217112
:1022F000E4FDFC121F0B0DBD00010CBC0DF5BD046F
:01230000F2EA
:0123010022B9
:0C233700C2867F057E00122171D2862232
:0A23580012218812232A43B120222B
:0923A10053B1DF1221C802232A06
:1018B80085423A854139854038853F37E53CB40152
:1018C80002C287122358E53E600302195C752201A3
:1018D800E47FE87E03FDFCAB3AAA39A938A837C3F0
:1018E8001206B74061E5226401705B7FDD7E03125A
:1018F8001C6C120C30E53A2418F53AE53934FCF53D
:1019080039E53834FFF538E53734FFF537E4FFFEBD
:10191800FDE537FC78181206C890E7C4EFF0E4FF3D
:10192800FEE538FDE4FC78101206C8A3EFF0E4FFEA
:10193800E539FEE4FDFC78081206C8A3EFF0E53AA5
:10194800FFA3EFF0808AE522B40112AE39AF3A1254
:101958001C6C8009752201E522640160FA1223A13A
:08196800E53CB40102D2872224
:101FF600AD07AC06D3ED9400EC9400401E00000043
:10200600EE90E6D0F0000000ED90E6D1F000000082
:0C20160075BB04000000E5BB30E7FB22B6
:081E34008C6E8D6FAB07AA064E
:101E3C00E4FDFCC3ED956FEC956E5022EA90E6D074
:101E4C00F0000000EB90E6D1F000000075BB05003F
:0E1E5C000000E5BB30E7FB0DBD00010C80D59A
:011E6A002255
:10207800AD07AC06000000ED25E0EC3390E6D0F0AB
:10208800000000ED25E090E6D1F000000075BB04EB
:09209800000000E5BB30E7FB226B
:10151500C20375450290E7C0E545F012233712185E
:10152500B81222F0121CB275450390E7C0E545F0EC
:101535003003030215DDE4F56CF56DC3E56D952803
:10154500E56C9527500D121F0B056DE56D70EC05CB
:101555006C80E8E53BD39400400CE53BFD7C00AF97
:1015650032AE31121E34D3E5249400E523940040B5
:1015750007AF24AE23122078E4F56AF56BC3E56B5B
:10158500954DE56A954C502C122022E4F56CF56DCD
:10159500C3E56D95337480F8656C98500D121F0B7B
:1015A500056DE56D70EA056C80E6056BE56B70CD44
:1015B500056A80C9E4F56CF56DC3E56D954AE56C82
:1015C5009549500D121F0B056DE56D70EC056C808E
:0815D500E8AF44AE43121FF61B
:0115DD0022EB
:10202200000000E53225E0E5313390E6D0F0000013
:1020320000E53225E090E6D1F000000075BB040017
:0B2042000000E5BB20E7033003F8229C
:1017E900E490E608F075C83443985053877FD2AC2B
:0717F90075CBFF75CA6422E5
:0D231000309902C2998F993099FDC299222F
:1020F00090000020981CA3AF82AE83E4FCFD7BFA25
:102100007AFFF9F8C31206A15004D2008004C2007D
:0621100080E1C298AF99C6
:0121160022A6
:1020A100E490E608F0D28E53897F5389BF4389209B
:1020B1005389EF438E10758DB243C05043D880C20F
:0820C100C0C2C1D2AED2AF22B1
:0D231D0030C102C2C18FC130C1FDC2C1225A
:1021170090000020C01CA3AF82AE83E4FCFD7BFAD5
:102127007AFFF9F8C31206A15004D2008004C20056
:0621370080E1C2C0AFC14F
:01213D00227F
:0423BE0075B00922CB
:0423C20075B00322CD
:0423C60075B00622C6
:072343007FC47E0912217125
:04234A0075B00C223C
:0D232A00E4F5B07525FF90E7CBE525F02226
:1021A90012216A1223BE12216D1223C212216D124D
:0F21B90023C6122163E4F52590E7CBE525F0223C
:1021C80012216A1223C612216D1223C212216D1226
:0F21D80023BE12216375250390E7CBE525F02286
:102188001223C27FC47E091221711223BE12234377
:102198007FC47E0912217175250190E7CBE525F0F2
:0121A8002214
:10204D001223BE7FC47E091221711223C27FC47E6A
:10205D00091221711223C61223437FC47E09122156
:0B206D007175250290E7CBE525F022FD
:0823B200E4F51DD2E9D2AF22CF
:101EA10090E678E020E6F9C2E990E678E04480F037
:101EB100EF25E090E679F090E678E030E0F990E601
:101EC10078E04440F090E678E020E6F990E678E0AA
:061ED10030E1D6D2E92247
:101F3D00A90790E678E020E6F9E51D702390E67894
:101F4D00E04480F0E925E090E679F08D18AF03A923
:101F5D00077519018A1A891BE4F51C751D01D32219
:021F6D00C3228D
:101ED700A90790E678E020E6F9E51D702590E678F9
:101EE700E04480F0E925E0440190E679F08D18AFF1
:101EF70003A9077519018A1A891BE4F51C751D03C7
:041F0700D322C322FC
:03004B000211653A
:10116500C0E0C083C082C085C084C086758600C0CB
:10117500D075D000C000C001C002C003C006C007C2
:1011850090E678E030E206751D0602124F90E6788B
:10119500E020E10CE51D64026006751D0702124F93
:1011A500E51D24FE605F14603624FE7003021240C4
:1011B50024FC700302124C2408600302124FAB1981
:1011C500AA1AA91BAF1C051C8F8275830012060382
:1011D50090E679F0E51C65187070751D05806B90BB
:1011E500E679E0AB19AA1AA91BAE1C8E827583009D
:1011F500120630751D02E5186401704E90E678E020
:101205004420F08045E51824FEB51C0790E678E0FB
:101215004420F0E51814B51C0A90E678E04440F047
:10122500751D0090E679E0AB19AA1AA91BAE1C8EB4
:1012350082758300120630051C800F90E678E04425
:1012450040F0751D008003751D005391DFD007D058
:1012550006D003D002D001D000D0D0D086D084D023
:0812650085D082D083D0E03275
:1021E700121ED7E51D24FA600E146006240770F34B
:0C21F700D322E4F51DD322E4F51DD32211
:10220300121F3DE51D24FA600E146006240770F3C7
:0C221300D322E4F51DD322E4F51DD322F4
:0300000002197072
:0C197000787FE4F6D8FD7581720219B78B
:10050D00E709F608DFFA8046E709F208DFFA803ED0
:10051D0088828C83E709F0A3DFFA8032E309F608BD
:10052D00DFFA8078E309F208DFFA807088828C8325
:10053D00E309F0A3DFFA806489828A83E0A3F608D9
:10054D00DFFA805889828A83E0A3F208DFFA804CB3
:10055D0080D280FA80C680D4806980F2803380108A
:10056D0080A680EA809A80A880DA80E280CA8033F3
:10057D0089828A83ECFAE493A3C8C582C8CCC5836B
:10058D00CCF0A3C8C582C8CCC583CCDFE9DEE7803B
:10059D000D89828A83E493A3F608DFF9ECFAA9F0BA
:1005AD00EDFB2289828A83ECFAE0A3C8C582C8CC10
:1005BD00C583CCF0A3C8C582C8CCC583CCDFEADE29
:1005CD00E880DB89828A83E493A3F208DFF980CC8B
:1005DD0088F0EF60010E4E60C388F0ED2402B40484
:1005ED000050B9F582EB2402B4040050AF2323452B
:0605FD00822390055D73EE
:10060300BB010CE58229F582E5833AF583E02250AC
:1006130006E92582F8E622BBFE06E92582F8E222F6
:0D062300E58229F582E5833AF583E4932210
:10063000F8BB010DE58229F582E5833AF583E8F000
:10064000225006E92582C8F622BBFE05E92582C8AC
:02065000F22294
:10065200E88FF0A4CC8BF0A42CFCE98EF0A42CFC47
:100662008AF0EDA42CFCEA8EF0A4CDA8F08BF0A4C5
:100672002DCC3825F0FDE98FF0A42CCD35F0FCEB24
:100682008EF0A4FEA9F0EB8FF0A4CFC5F02ECD39E9
:0F069200FEE43CFCEAA42DCE35F0FDE43CFC2256
:101CF800C2D5E830E70FB2D5E4C39BFBE49AFAE417
:101D080099F9E498F8EC30E717B2D5121D2E1207AE
:101D18007DE4C39BFBE49AFAE499F9E498F880031C
:101D280012077D30D50DE4C39FFFE49EFEE49DFDC0
:041D3800E49CFC2209
:1006A100EB9FF5F0EA9E42F0E99D42F0EC6480C8D0
:0606B10064809845F02270
:1006B700EB9FF5F0EA9E42F0E99D42F0E89C45F099
:0106C7002210
:1006C800E8600FECC313FCED13FDEE13FEEF13FF10
:0306D800D8F12234
:1006DB00E86010ECA2E713FCED13FDEE13FEEF1335
:0406EB00FFD8F02222
:1006EF00D083D082F8E4937012740193700DA3A39A
:1006FF0093F8740193F5828883E4737402936860AE
:06070F00EFA3A3A380DFAD
:10071500EF4E6012EF60010EEDBB010B89828A83FB
:10072500F0A3DFFCDEFA2289F05007F709DFFCA908
:0C073500F022BBFEFCF309DFFCA9F0225F
:10197C00020FB8E493A3F8E493A34003F68001F2BA
:10198C0008DFF48029E493A3F85407240CC8C3336C
:10199C00C4540F4420C8834004F456800146F6DF3B
:1019AC00E4800B010204081020408090136AE47E4E
:1019BC00019360BCA3FF543F30E509541FFEE49330
:1019CC00A360010ECF54C025E060A840B8E493A3F7
:1019DC00FAE493A3F8E493A3C8C582C8CAC583CA22
:1019EC00F0A3C8C582C8CAC583CADFE9DEE780BEDA
:01144A0000A1
:1007410075F008758200EF2FFFEE33FECD33CDCC6F
:1007510033CCC58233C5829BED9AEC99E5829840F2
:100761000CF582EE9BFEED9AFDEC99FC0FD5F0D6CF
:10077100E4CEFBE4CDFAE4CCF9A88222B800C1B9F9
:100781000059BA002DEC8BF084CFCECDFCE5F0CB37
:10079100F97818EF2FFFEE33FEED33FDEC33FCEB70
:1007A10033FB10D703994004EB99FB0FD8E5E4F92B
:1007B100FA227818EF2FFFEE33FEED33FDEC33FC18
:1007C100C933C910D7059BE99A4007EC9BFCE99A0C
:1007D100F90FD8E0E4C9FAE4CCFB2275F010EF2F51
:1007E100FFEE33FEED33FDCC33CCC833C810D70751
:1007F1009BEC9AE899400AED9BFDEC9AFCE899F88C
:0E0801000FD5F0DAE4CDFBE4CCFAE4C8F9221E
:00000001FF
